:100000007428A800F839A000A00CA00C200C8407CC
:100010001320A80000056F282808031C0301000610
:10002000280580066F2800308A00280807398207D3
:100030000134023404340834103420344034803421
:10004000A301A200FF30A207031CA307031C6F2813
:100050000330A100DF302E202228A101E83EA000BD
:10006000A109FC30031C3728A00703183428A00777
:100070006400A10F342820183D28A01C412800004E
:10008000412808000310A00DA10DFF3E03184228CF
:1000900020086F28A101A301A20001305428A1016A
:1000A000A301A20004305428A80023082102031D44
:1000B0005B282208200204300318013003190230A3
:1000C0002805031DFF306F280038031DFF3004058D
:1000D000031DFF306F280404031DFF306F288313B6
:1000E000031383126400080007309F000330A3004D
:1000F000E8308A0121208316860185018312C6011A
:10010000C001BF018A11A6284508123C031DFF301B
:10011000FF3ABA004508593C031DFF30FF3ABC00C6
:100120003A0884003C088A016B20BC00BD006400D2
:100130003C083D048A1103199E28C6016400450845
:10014000143C8A11031DA528C001C201C5018316F4
:1001500085140514831264008A110518B1288A01D8
:10016000AB2864008A11051CB7288A01B128C10197
:1001700064000A3041028A110318D32864008A11EE
:100180000518C4288A01BE28383084004108003E82
:100190008A0101200310851803148A010C20C10A6A
:1001A0008A11031DB8280730C1000310C50D38306F
:1001B00084004108003E8A0101200030031D013007
:1001C000BA00BB013A08C5070130C1028A11031801
:1001D000D528831605108312051064004208023CDE
:1001E0008A11031DF5288A01842864004508F03C23
:1001F0008A11031DFF280230C2008A01A628450883
:10020000123C031DFF30FF3ABA004508593C031D5C
:10021000FF30FF3ABC003A0884003C088A016B209A
:10022000BC00BD0064003C083D048A1103191C2970
:100230008030C6008A01A62864004508583C8A110F
:10024000031D26298A1160228A01A6286400450818
:10025000E03C8A11031D2E298A01A6286400450866
:10026000143C8A11031D38290230C0008A01A628D7
:10027000640045085A3C8A11031D42290D30BE0016
:100280008A11512A4608C507FF30C300FF30A2007B
:10029000A20A22085F3C8A11031CBC298A1158213A
:1002A00045028A11031D48292208C3008A11BC296E
:1002B00001308A0022088207293496349E345D3446
:1002C000A534AE34BD345234C634C534BE34D5340E
:1002D00041344E3449344A34453416341E342634BD
:1002E00025342E3436343D343E344634CC344C340C
:1002F000C1345534C934CA34D2349C34B234A134F4
:10030000A334A434AB34B434B334C334BB34C234B4
:10031000CB34BA34B134C434CD349534AD349B3499
:10032000AC34BC34AA349D34A234B5349A34543439
:1003300061345B34B634CE34A6341C3432342134C8
:10034000233424342B343434333443343B34423474
:100350004B343A34313444344D3415342D341B3459
:100360002C343C342A341D34223435341A34D434F9
:10037000E134DB34DD34663464004308FF3C8A1129
:10038000031DC4298A11002A64004008023C8A1116
:10039000031DCF2940304302BE008A11512A640058
:1003A0003F08003C8A11031DD7298A114E2A4308B1
:1003B000A00040308A014A20BA004308A0005B3008
:1003C0008A014F20BC003A0884003C088A0164205E
:1003D000BC00BD0064003C083D048A110319F429E7
:1003E0004308BE008A11512A640043081B3C8A114D
:1003F000031DFE293A30BE008A11512A8A114E2A65
:10040000FF30A200A20A22080F3C8A11031C262AF0
:100410008A11122245028A11031D022A2208C300F2
:100420008A11262A02308A00220882077034693431
:1004300072347A346B34733474346C3475347D3480
:100440007C347B34793471340D3476346400430861
:10045000FF3C8A11031D2E2A8A01A62843080F3C5F
:100460008A11031C4C2A8A113822BE008A114C2A98
:1004700002308A0043088207303431343234333456
:100480003434353436343734383439342A342D342E
:100490002B342E3409341B348A11512A203043075F
:1004A000BE00861702308A0120203E0886000230F6
:1004B0008A01202086178A01A62863008A015D2A06
:1004C00064003F08003C8A11031D6A2A0430BF0003
:0804D0008A116B2ABF0108002C
:02400E007C3FF5
:00000001FF
